:100000000C9466020C94AD020C94AD020C94AD02FB
:100010000C94AD020C94AD020C94AD020C94AD02A4
:100020000C94AD020C94AD020C94CF0B0C94A10C6B
:100030000C94AD020C94AD020C94AD020C94AD0284
:100040000C94AD020C9415210C94AD020C94AD02ED
:100050000C94AD020C94A71A0C94AD020C94AD0252
:100060000C94AD020C94AD020C94AD020C94AD0254
:100070000C94AD020C94AD020C94AD020C94AD0244
:100080000C94AD020C94AD020C94AD020C94AD0234
:100090000C94AD020C94AD020C94AD020C94AD0224
:1000A0000C94AD020C94AD020C94AD020E0D300D0B
:1000B000230E300D230E750D980D230EED0D000E41
:1000C000EA10EA10191119115C119611A313A31368
:1000D000AF11A313A412A4127713A313A3138E13A7
:1000E0000000F0A1F0A329002B000354E1003581AA
:1000F00000001E00140004001D7164004D001F006C
:100100001A0016001B00E1044C0020000800070044
:10011000060050002A0021001500090019004F00B8
:100120004A00220017000A000500000002541908C6
:10013000E3000000E20000002E770608E700000060
:10014000E60000002E7F23001C000B0011000000C1
:100150000454240018000D00100052004B0025002C
:100160000C000E00360051002C00260012000F007B
:100170003700E108280027001300330038713000F1
:100180004E002D002F003482E50031810000010077
:100190000100010001000100000001000100010058
:1001A00001000100010001000100500001000100F8
:1001B0000100010052005100010001000100010096
:1001C00001004F00010001000100010001000100D9
:1001D000010000000100010001000000010000001A
:1001E00001000100010000000100000001003F00CB
:1001F00052005100230200000100400024002100B1
:100200001E00270001004100250022001F003700CA
:1002100001004200260023002000270001004300C7
:100220003002300024022E0001004400450001008D
:1002300001000100000001000100010001000100B7
:100240000000010001000100FB00010001000100AD
:100250000100F200F900010001000100F000F100CE
:10026000FA00F400010001000100F300FC00F500B9
:100270000100010001000100F60000000100010082
:100280000100000001000000010001000100000069
:100290000100000001000100010001000100000058
:1002A0000100010001000100A800A90001000100F7
:1002B00001000100AC00AA00B6000100010001002D
:1002C000AB0050000100010001000100520051008C
:1002D0000100AE000100010001004F000000160304
:1002E0004500720067006F0044006F007800200036
:1002F00045005A00000016034500720067006F00B9
:1003000044006F007800200045005A0000000403FC
:10031000090409026D00040100A0FA0904000001AB
:1003200003010100092111010001223F000705819D
:100330000308000A09040100010301020009211158
:10034000010001224D000705820308000A0904028A
:1003500000010300000009211101000122360007FD
:1003600005830308000A09040300010300000009D3
:100370002111010001223900070584031000011238
:1003800001100100000008EDFE071301000102004A
:100390000105010906A101050719E029E715002556
:1003A0000195087501810205081901290595057552
:1003B000019102950175039101050719002977152F
:1003C000002501957875018102C005010980A10110
:1003D000850216010026B7001A01002AB700751021
:1003E00095018100C0050C0901A1018503160100DA
:1003F000269C021A01002A9C02751095018100C0FA
:1004000005010902A1010901A10005091901290538
:10041000150025019505750181029501750381017E
:100420000501093009311581257F9502750881067E
:1004300009381581257F950175088106050C0A3854
:10044000021581257F950175088106C0C005010947
:1004500006A101050719E029E71500250195087592
:100460000181029501750881010508190129059589
:100470000575019102950175039101050719002980
:10048000FF150025FF950675088100C000000000DB
:1004900000000000000000010204060A0F17202CD3
:1004A0003A4A5D71879DB3C7DAE9F5FCFFFCF5E9CF
:1004B000DAC7B39D87715D4A3A2C20170F0A0604EC
:1004C00002010000000000000000000011241FBE17
:1004D000CFEFDAE0DEBFCDBF04B603FE27C08091C8
:1004E000ED019091EE01A091EF01B091F001873004
:1004F000904BA740B04BD1F41092ED011092EE0159
:100500001092EF011092F00114BE84B7877F84BF70
:100510000FB6F894A8958091600088618093600080
:10052000109260000FBEE0E0FFE3099511E0A0E04B
:10053000B1E0ECECF5E402C005900D92A433B107F4
:10054000D9F721E0A4E3B1E001C01D92AD3EB207AE
:10055000E1F70E9416090C94E4220C94000061114A
:100560000BC0FC018281882321F085EE0E94840F5C
:1005700003C085EE0E944C1080E090E0089508953D
:100580006091B1017091B2018091B3019091B40179
:100590000E94D41956985E9825982D9826982E98E2
:1005A00027982F98823061F018F4813031F0089547
:1005B000833059F0843039F00895259A2D9A0895A2
:1005C000269A2E9A0895259A2D9A279A2F9A089559
:1005D0000C94C00256985E9825982D9826982E98CF
:1005E00027982F988FEF90E0909389008093880050
:1005F00090938B0080938A0090938D0080938C0061
:10060000259A2D9A2FEF80E792E02150804090406C
:10061000E1F700C00000269A2E9A2FEF80E792E0C3
:10062000215080409040E1F700C00000279A2F9AA7
:100630002FEF80E792E0215080409040E1F700C02A
:10064000000025982D982FEF80E792E02150804000
:100650009040E1F700C0000026982E982FEF80E729
:1006600092E0215080409040E1F700C000002798C0
:100670002F9856985E9825982D9826982E9827980A
:100680002F98089589EA8093800089E08093810003
:1006900024982C983F988AB18F748AB96E98479A9B
:1006A0008BB1806B8BB9769A0E94EA020C94BF02E0
:1006B00080E2809300018091340181110EC00E947C
:1006C000A70381E0809334012FEF83ED90E3215065
:1006D00080409040E1F700C0000080E40E94AD033C
:1006E0008093000181112EC00E94D70380930001E6
:1006F000811128C00E94D70380930001811122C07C
:100700008FE30E94D7038093000181111BC00E94D8
:10071000CF0380E40E94AD0380930001811112C0D9
:100720008CE00E94D7038093000181110BC00E94CE
:10073000D70380930001811105C08FE30E94D70386
:10074000809300010E94CF038091000108951092D0
:10075000B9008AE08093B800089594EA9093BC00B1
:100760009091BC0097FFFCCF9091B900987F983092
:1007700021F0903111F081E008958093BB0084E86E
:100780008093BC008091BC0087FFFCCF8091B900B2
:10079000887F883111F0803471F780E0089584E912
:1007A0008093BC008091BC0084FDFCCF08958093B1
:1007B000BB0084E88093BC008091BC0087FFFCCF25
:1007C0009091B900987F81E0983209F480E0089513
:1007D00084E88093BC008091BC0087FFFCCF8091AF
:1007E000BB00089580910001811115C080E40E9432
:1007F000AD038093000181110CC082E10E94D703F8
:1008000080930001811105C08FEF0E94D703809370
:1008100000010E94CF0384B1807F84B985B1807FBD
:1008200085B98AB1837F8AB98BB1837F8BB93E98B2
:10083000469808950E945803809300010E94F20395
:1008400080B38C7080BB81B3836F81BBE4E4F1E043
:10085000A6E3B1E011921D9281E0E235F807D1F7ED
:100860000C9442039F92AF92BF92CF92DF92EF928D
:10087000FF920F931F93CF93DF9380910001882302
:1008800079F0809135018F5F80933501811108C027
:100890000E94580380930001811102C00E94EA0265
:1008A00086E3E82E81E0F82E8701C0E0D0E0BB248B
:1008B000B39492E0A92ECC24C394D12CC730D10597
:1008C00000F580910001811164C080E40E94AD03B5
:1008D00080930001811112C082E10E94D7038093AE
:1008E000000181110BC0C6010C2E01C0880F0A94B3
:1008F000EAF780950E94D703809300010E94CF03FE
:1009000048C0CA30A1F028F4C83059F0C93061F0AD
:1009100005C0CC3089F070F0CD3089F0209A28984D
:1009200010C0219A29980DC0229A2A980AC0239AA9
:100930002B9807C0529A01C0539A5B9802C03E9A06
:100940004698E0EAEA95F1F78FB181708B257999A5
:1009500002C032E001C030E0832B7C9902C034E059
:1009600001C030E0832B7D9902C028E001C020E067
:10097000822B7E9902C090E101C090E0892B9FB14B
:100980009095991F9927991F9295990F907E892B81
:100990000FC08091000181114AC080E40E94AD0324
:1009A00080930001882381F1912C0E94CF03892D2F
:1009B000D8019C91981719F08C93A09201010E9484
:1009C000F20321960F5F1F4FCE30D10509F076CF8D
:1009D00080910101882369F181508093010188236E
:1009E00039F0EFE9FFE03197F1F700C0000021C0D6
:1009F000E4E4F1E0D7018D917D018193B4E4EB163D
:100A0000B1E0FB06B9F715C083E10E94D7038093DC
:100A100000018111C9CF81E40E94AD0380930001E0
:100A20008111C2CF0E94E803982E9094BECF80E03F
:100A3000BFCF0E94E80281E0DF91CF911F910F911B
:100A4000FF90EF90DF90CF90BF90AF909F90089570
:100A5000E82FF0E0EC5BFE4F8081089508958B3B1A
:100A6000910580F4883A910548F5853A9105D8F4C6
:100A70008430910508F0B2C0019709F06EC081E0A2
:100A800090E00895803E910508F467C0883E910586
:100A900008F4A4C09C01205F31092031310508F021
:100AA0005CC090650895853A910509F459C0863A6D
:100AB000910509F058C082E890E40895883A9105BC
:100AC00009F454C0893A910509F453C08A3A910552
:100AD00009F452C08B3A910509F451C08C3A910542
:100AE00009F450C08D3A910509F44FC0803B91053F
:100AF00009F44EC08E3A910509F44DC08F3A910524
:100B000009F44CC0813B910509F44BC0823B91052F
:100B100009F44AC0833B910509F449C0843B91051F
:100B200009F448C0853B910509F447C0863B91050F
:100B300009F446C0873B910509F445C0883B9105FF
:100B400009F444C0893B910509F443C08A3B9105EF
:100B500009F442C080E094E4089580E090E00895B4
:100B600081E890E4089583E890E4089582EE94E4A7
:100B7000089589EE94E408958AEE94E4089585EB4F
:100B800094E4089586EB94E4089587EB94E4089543
:100B90008CEC94E408958DEC94E4089583E895E456
:100BA00008958AE895E4089582E995E4089584E932
:100BB00095E4089581E296E4089583E296E4089529
:100BC00084E296E4089585E296E4089586E296E448
:100BD000089587E296E408958AE296E408950895D8
:100BE00024E5829FC0011124FC0126E0729FE00DE4
:100BF000F11D1124E60FF11DEE0FFF1FEA51FF4F0B
:100C0000859194910895880F991FFC01E05AF04056
:100C1000859194910895880F991FFC01E052FF4F30
:100C200085919491089524E5829FC0011124FC01CF
:100C300046E0749FE00DF11D1124E60FF11DEE0F4B
:100C4000FF1FEA51FF4F859194919C013A95211520
:100C50004FE1340708F425C13F512115304120F4FC
:100C60009F700E940B0608959C013053211530415E
:100C700018F49927906C0895811520E5920769F47E
:100C80000E94C5134FEF84E39CE0415080409040A8
:100C9000E1F700C000000C94CC1A813020E59207E7
:100CA00031F48091CC0181608093CC0108959C0146
:100CB00030552115304108F05CC0292F33272F70A3
:100CC000332721303105E9F4AC0164E0440F551FAE
:100CD0006A95E1F744275370BC016370772702C01F
:100CE000220F331F6A95E2F73C68242B352B73E003
:100CF000880F991F7A95E1F780769927822B932B9D
:100D000008952230310529F4982F8827816F906A41
:100D1000089523303105A1F4AC0133E0440F551F91
:100D20003A95E1F7407E57708370992721E030E0D3
:100D300002C0220F331F8A95E2F7C9019C6816C0D2
:100D40002430310531F5AC0123E0440F551F2A95BD
:100D5000E1F7407E57708370992721E030E002C0B0
:100D6000220F331F8A95E2F7C9019A68842B952BCD
:100D700008959C0130572115304118F49F709062FE
:100D800008959C0130582115304118F49F70906AE5
:100D90000895803E9105E0F4803C910558F581333B
:100DA000910509F46FC048F48932910509F463C0D4
:100DB0008A32910509F46DC072C089339105E9F05A
:100DC00082389105D1F08533910509F44DC067C093
:100DD000833E910581F138F4803E9105B9F0823E61
:100DE0009105D9F05CC0863E910561F1873E910581
:100DF000A1F155C00E94030608952091DE0120FD57
:100E000002C021FF4CC080EE90E049C08091DE011D
:100E100080FFF9CF89E390E042C08091DE0182FF3C
:100E20000EC08091DE0184FF03C080E090E037C0F7
:100E300083EE90E034C08091DE0182FFF2CF82EE3B
:100E400090E02DC08091DE0183FF0BC08091DE0118
:100E500084FDEBCF87EE90E022C08091DE0183FF1E
:100E6000F5CF86EE90E01BC08091DE0185FF07C0C4
:100E700089E290E014C08091DE0185FFF9CF85E31F
:100E800090E00DC08091DE0186FF07C08AE290E00D
:100E900006C08091DE0186FFF9CF81E390E00E94D9
:100EA0002F0508950895809162010895CF93DF93EF
:100EB00000D01F92CDB7DEB79C018091E401843051
:100EC00019F593E099833B832A839093E9008FEF90
:100ED0009091E800815095FD06C095ED9A95F1F747
:100EE00000008111F5CF8091E80085FF0DC040E042
:100EF00050E063E070E0CE0101960E94C30980914A
:100F0000E8008E778093E8000F900F900F90DF91AC
:100F1000CF910895CF93DF9300D01F92CDB7DEB766
:100F20002091E401243021F522E029839B838A83E8
:100F300083E08093E9008FEF9091E800815095FD68
:100F400006C095ED9A95F1F700008111F5CF8091DB
:100F5000E80085FF0DC040E050E063E070E0CE01A6
:100F600001960E94C3098091E8008E778093E80083
:100F70000F900F900F90DF91CF9108959C01809179
:100F8000E4018430F9F482E08093E9009FEF8091DE
:100F9000E800915085FD06C085ED8A95F1F70000C7
:100FA0009111F5CF8091E80085FF0CC040E050E042
:100FB00065E070E0C9010E94C3098091E8008E7766
:100FC0008093E8000895CF93DF93EC018091E401D2
:100FD000843009F046C090910C019923D9F090918A
:100FE0000D019923B9F08093E9008FEF9091E8000B
:100FF000815095FD06C095E19A95F1F700008111A9
:10100000F5CF8091E80085FF2CC040E050E060E122
:1010100070E017C081E08093E9008FEF9091E800C5
:10102000815095FD06C095ED9A95F1F7000081116C
:10103000F5CF8091E80085FF14C040E050E068E003
:1010400070E0CE010E94C3098091E8008E77809302
:10105000E80080E1FE01A2E5B1E001900D928A95E1
:10106000E1F7DF91CF9108958091E301811109C0EB
:101070000E94540B0E94B10B8091E2008460809327
:10108000E20008951092E301089508950C9402215E
:101090000E94621A0E9408210E945C0E0C94520762
:1010A00042E061EC81E00E94CD0A42E061EC82E026
:1010B0000E94CD0A42E061EC83E00E94CD0A42E149
:1010C00061EC84E00C94CD0A8091E601833009F450
:1010D00055C030F4813071F0823009F48EC008952B
:1010E0008A3009F47AC08B3009F460C0893009F085
:1010F0009CC020C08091E501813A09F096C08091A2
:10110000E800877F8093E8008091E9019091EA01EF
:10111000892B21F460E182E591E003C060E080E08A
:1011200090E070E00E940E0A8091E8008B77809337
:10113000E80008958091E501813209F076C0809140
:10114000E9019091EA01009719F0039709F06DC049
:101150008091E800877F8093E8008091E80082FD1D
:1011600005C08091E4018111F8CF5FC08091F1004A
:10117000809362018091E8008B7753C08091E501F4
:10118000813A09F052C08091E9019091EA01892BDE
:1011900009F04BC08091E800877F8093E800809140
:1011A000E80080FFFCCF80910C0136C08091E50102
:1011B0008132D9F58091E9019091EA01892BA9F555
:1011C0008091E800877F8093E8000E94020B809165
:1011D000E70180930C010C94C5138091E5018132E5
:1011E00021F58091E800877F8093E8000E94020B40
:1011F0008091E8018093630108958091E501813A2F
:10120000A1F48091E800877F8093E8008091E80056
:1012100080FFFCCF809163018093F1008091E80012
:101220008E778093E8000C94020B089584B7877F33
:1012300084BF0FB6F894A895809160008861809370
:101240006000109260000FBE90E080E80FB6F89446
:1012500080936100909361000FBE0E94AB0E0E94CC
:10126000540B0E94B10B8091E20084608093E200F5
:1012700078940E943C0E0E94AD0E82E091E00E94A4
:10128000570E0E94F0208091E401853069F40E949D
:10129000241A8091E2018823B1F30E944E1A882318
:1012A00091F30E94AD09EFCF0E94B30EECCF292F2E
:1012B000332723303105C9F060F42130310581F046
:1012C0002230310509F041C08DE690E022E133E0A3
:1012D00040C021323105E1F02232310531F135C013
:1012E00082E190E02FE733E034C099278130910507
:1012F00049F028F0029749F5EEEDF2E005C0EEE086
:10130000F3E002C0E6EFF2E0849190E09F0121C09B
:101310006430D8F4E62FF0E0EE0FFF1FEE5DFE4FD5
:101320002081318189E090E014C0643070F470E075
:10133000FB01EE0FFF1FE65EFE4F20813181FB01B6
:10134000EA5EFE4F808190E004C080E090E020E003
:1013500030E0FA0131832083089580E189BD82E184
:1013600089BD09B400FEFDCF8091D8008F7D8093A8
:10137000D8008091E00082608093E0008091E000DE
:1013800081FDFCCF0895CF92DF92EF92FF920F93F1
:101390001F93CF93DF93EC018B016A010E94210B15
:1013A000811133C0C114D10439F0F60180819181DB
:1013B000081B190BC80FD91FE12CF12C01151105C1
:1013C00019F18091E80085FD16C08091E8008E77C4
:1013D0008093E800C114D10449F0F6018081918125
:1013E000E80EF91EF182E08285E00FC00E94210B19
:1013F000882321F30AC089918093F10001501109DB
:10140000FFEFEF1AFF0ADACF80E0DF91CF911F9153
:101410000F91FF90EF90DF90CF9008952091EB0116
:101420003091EC012617370748F06115710539F442
:101430002091E8002E772093E80001C0B901FC015B
:1014400020E06115710579F18091E4018823F1F1C3
:101450008530F1F18091E80083FD3CC08091E80087
:1014600082FD2EC08091E80080FFEBCF2091F30039
:101470008091F20090E0922B6115710551F0883057
:10148000910538F421912093F10061507109019682
:10149000F3CF21E0089709F020E08091E8008E77F3
:1014A0008093E800CECF2111CFCF0AC08091E40114
:1014B000882361F0853061F08091E80083FD0AC0E7
:1014C0008091E80082FFF2CF80E0089582E00895E5
:1014D00083E0089581E008952091EB013091EC01C3
:1014E0002617370748F06115710539F42091E80097
:1014F0002E772093E80001C0B901FC0120E06115BE
:10150000710591F18091E401882309F440C0853090
:1015100009F43FC08091E80083FD3DC08091E80060
:1015200082FD2FC08091E80080FFE9CF2091F30079
:101530008091F20090E0922B6115710559F088308E
:10154000910540F424912093F10031966150710986
:101550000196F2CF21E0089709F020E08091E800A1
:101560008E778093E800CBCF2111CCCF0AC0809139
:10157000E401882361F0853061F08091E80083FD0B
:101580000AC08091E80082FFF2CF80E0089582E0F7
:10159000089583E0089581E00895982F973068F5C5
:1015A0009093E900981739F07091EC002091ED00CC
:1015B0005091F00003C0242F762F50E021FD02C08F
:1015C0009F5FECCF3091EB003E7F3093EB0030918A
:1015D000ED003D7F3093ED003091EB0031603093B2
:1015E000EB007093EC002093ED005093F0002091FD
:1015F000EE0027FDE5CF80E008958F708093E9002D
:1016000081E008958091E50187FF11C08091E80095
:1016100082FD05C08091E4018111F8CF11C0809155
:10162000E8008B770BC08091E401882349F080911A
:10163000E80080FFF8CF8091E8008E778093E80083
:1016400008952091E4003091E50095E64091EC008A
:10165000842F817040FF23C08091E80080FD1DC071
:101660008091E401882399F0853099F08091EB0016
:1016700085FD11C04091E4005091E5002417350725
:1016800029F3915011F09A01E1CF84E0089582E0AE
:10169000089583E0089581E0089580E008954091E1
:1016A000E80042FFDDCF08950E94C20B0E94CA0BE2
:1016B000E0EEF0E0808181608083E8EDF0E0808101
:1016C0008F77808319BCA7EDB0E08C918E7F8C93CF
:1016D00080818F7E80831092E30108950F931F9382
:1016E000CF93DF930E94C20B0E94CA0BC8EDD0E0DB
:1016F00088818F77888388818068888388818F7DBF
:10170000888319BC1092E4011092E0011092E2016A
:101710001092E10100EE10E0F80180818B7F808360
:1017200088818160888342E060E080E00E94CD0A89
:10173000E1EEF0E080818E7F8083E2EEF0E0808158
:1017400081608083808188608083F80180818E7FC2
:101750008083888180618883DF91CF911F910F9171
:101760000895E8EDF0E080818F7E8083E7EDF0E082
:1017700080818160808384E082BF81E08093E30187
:101780000C946E0BE8EDF0E080818E7F80831092E8
:10179000E20008951092DA001092E10008951F927D
:1017A0000F920FB60F9211242F933F934F935F9395
:1017B0006F937F938F939F93AF93BF93EF93FF9319
:1017C0008091E10082FF0BC08091E20082FF07C0A0
:1017D0008091E1008B7F8093E1000E943B0E80911D
:1017E000DA0080FF1FC08091D80080FF1BC080916D
:1017F000DA008E7F8093DA008091D90080FF0DC0DF
:1018000080E189BD82E189BD09B400FEFDCF81E0A0
:101810008093E4010E94340805C019BC1092E401D1
:101820000E9442088091E10080FF19C08091E2008F
:1018300080FF15C08091E2008E7F8093E20080914E
:10184000E20080618093E2008091D8008062809302
:10185000D80019BC85E08093E4010E94460880917D
:10186000E10084FF30C08091E20084FF2CC080E161
:1018700089BD82E189BD09B400FEFDCF8091D80009
:101880008F7D8093D8008091E1008F7E8093E1006E
:101890008091E2008F7E8093E2008091E20081607F
:1018A0008093E2008091E001882311F084E007C07A
:1018B0008091E30087FD02C081E001C083E0809356
:1018C000E4010E9448088091E10083FF29C08091D3
:1018D000E20083FF25C08091E100877F8093E100D3
:1018E00082E08093E4011092E0018091E1008E7F1C
:1018F0008093E1008091E2008E7F8093E2008091EE
:10190000E20080618093E20042E060E080E00E94BB
:10191000CD0A8091F00088608093F0000E94450815
:10192000FF91EF91BF91AF919F918F917F916F91B7
:101930005F914F913F912F910F900FBE0F901F908D
:1019400018951F920F920FB60F9211242F933F9369
:101950004F935F936F937F938F939F93AF93BF93B7
:10196000CF93DF93EF93FF93C091E900CF70809105
:10197000EC00D82FD17080FDD0E81092E900809162
:10198000F000877F8093F00078940E94E50C10921D
:10199000E9008091F00088608093F000CD2BCF703B
:1019A000C093E900FF91EF91DF91CF91BF91AF918B
:1019B0009F918F917F916F915F914F913F912F9167
:1019C0000F900FBE0F901F9018951F93CF93DF932A
:1019D000CDB7DEB7AA970FB6F894DEBF0FBECDBF66
:1019E000E5EEF1E08091F100819321E0ED3EF20718
:1019F000C9F70E9464088091E80083FF24C18091A8
:101A0000E5019091E601492F50E04A30510508F078
:101A10001AC1FA01EA5AFF4F0C949922803881F0DA
:101A2000823809F010C18091E9018F708093E9003C
:101A30008091EB0085FB882780F91092E90006C0B1
:101A40008091E1019091E201911182609091E80012
:101A5000977F9093E8008093F1001092F100C8C046
:101A6000282F2D7F09F0EFC0882319F0823061F014
:101A7000EAC08091E701813009F0E5C0933009F0B8
:101A800080E08093E2012BC08091E701811127C0A3
:101A90008091E9018F7009F4D6C08093E90020910C
:101AA000EB0020FF1CC0933021F48091EB0080629A
:101AB00014C09091EB0090619093EB0021E030E036
:101AC000A90102C0440F551F8A95E2F74093EA002E
:101AD0001092EA008091EB0088608093EB001092F6
:101AE000E9008091E800877F86C08111ACC0109129
:101AF000E7011F778091E3008078812B8093E300DA
:101B00008091E800877F8093E8000E94020B80911B
:101B1000E80080FFFCCF8091E30080688093E300C1
:101B2000111102C082E001C083E08093E4018BC008
:101B30008058823008F087C08091E7019091E801D9
:101B40008C3D53E0950779F583E08A838AE28983A7
:101B50004FB7F894DE01139620E03EE051E2E32F08
:101B6000F0E050935700E49120FF03C0E295EF703E
:101B70003F5FEF708E2F90E0EA3010F0C79601C003
:101B8000C0968D939D932F5F243149F74FBF80916D
:101B9000E800877F8093E8006AE270E0CE0101965A
:101BA0000E940E0A14C0AE014F5F5F4F6091E901C1
:101BB0000E945709BC01892B09F445C09091E800A7
:101BC000977F9093E80089819A810E946C0A8091A6
:101BD000E8008B778093E80036C08038A1F58091CB
:101BE000E800877F8093E8008091E0018093F10016
:101BF0008091E8008E778093E8000E94020B23C05A
:101C0000811121C08091E7019091E8019927029705
:101C1000D4F48091E800877F8093E8008091E70109
:101C20008093E0010E94020B8091E001811106C0C7
:101C30008091E30087FD02C081E001C084E08093D1
:101C4000E4010E9450088091E80083FF0AC080915F
:101C5000E800877F8093E8008091EB0080628093AA
:101C6000EB00AA960FB6F894DEBF0FBECDBFDF9192
:101C7000CF911F9108950895CF938091E401882317
:101C8000A1F0C091E900CF709091EC00892F817094
:101C900090FD80E8C82B1092E9008091E80083FD58
:101CA0000E94E50CCF70C093E900CF910895909306
:101CB0006901809368010895E0916801F0916901DC
:101CC000309721F00190F081E02D099480E0089593
:101CD000E0916801F0916901309721F00280F38171
:101CE000E02D09940895E0916801F0916901309721
:101CF00021F00480F581E02D09940895209166017A
:101D0000309167012817390771F09093670180932C
:101D10006601E0916801F0916901309721F0068039
:101D2000F781E02D099408952091640130916501B7
:101D30002817390771F09093650180936401E09151
:101D40006801F0916901309721F00084F185E02D60
:101D50000994089508950C94AA0E0E94681A0E948E
:101D60001A040C942E1BCF92DF92EF92FF920F93E6
:101D70001F93CF93DF93CDB7DEB72B970FB6F894B1
:101D8000DEBF0FBECDBF0E9432048BE6C82E81E0BD
:101D9000D82E00E010E0E02E802F0E942805F601EA
:101DA00041916F01F82EF426B1F40F5F1F4F0E30F2
:101DB000110589F78FEF89838A831B820E94711A2C
:101DC0008160782F9D838C8349815A816B818D81BD
:101DD0000E94560F40C09091CC0191FF04C08B87A8
:101DE0000E942E058B8520E030E04F2D50E0922F91
:101DF000BA01022E02C0759567950A94E2F760FF5A
:101E000024C02E83EF8221E030E0690102C0CC0CB7
:101E1000DD1C9A95E2F790E08C219D21892B09F435
:101E200020E028870E94711A8160782F9A8789871D
:101E30004E815F8168858A850E94560FF801E559B9
:101E4000FE4F8081C826C08206C02F5F3F4F2630DC
:101E5000310569F6AACF0E94151E0E945C0E909172
:101E60006A018917A1F00E945C0E80936A012B968B
:101E70000FB6F894DEBF0FBECDBFDF91CF911F919B
:101E80000F91FF90EF90DF90CF900C9452072B961C
:101E90000FB6F894DEBF0FBECDBFDF91CF911F917B
:101EA0000F91FF90EF90DF90CF900895CF93DF9345
:101EB000CDB7DEB72B970FB6F894DEBF0FBECDBF00
:101EC0004F83588769877A878B87DE01119686E072
:101ED000FD0111928A95E9F785E0FE0137960190A0
:101EE0000D928A95E1F749815A816B817C818D81C0
:101EF0009E810E9459162B960FB6F894DEBF0FBE36
:101F0000CDBFDF91CF910895CF93C82F882309F4D7
:101F1000C1C0823859F40E945C0E81FDBBC089E3C8
:101F20000E94F6180E94AE1989E30CC0833879F438
:101F30000E945C0E80FDAEC083E50E94F6180E94F0
:101F4000AE1983E50E943519CF910C94AE198438EF
:101F500059F40E945C0E82FD9DC087E40E94F61831
:101F60000E94AE1987E4EECF8CEF8C0F813A48F4D3
:101F70008C2F0E94552081118DC08C2F0E94F61845
:101F8000E3CF80E28C0F883048F4C77081E001C055
:101F9000880FCA95EAF70E947719D6CF8BE58C0F88
:101FA000833078F4C53A29F0C63A31F083E890E0FE
:101FB00005C081E890E002C082E890E0CF910C94E7
:101FC0007E0E88E58C0F833108F064C0C83A39F181
:101FD000C93A41F1CA3A49F1CB3A51F1CC3A59F1F7
:101FE000CD3A61F1C03B69F1CE3A71F1CF3A79F166
:101FF000C13B81F1C23B89F1C33B91F1C43B99F1F3
:10200000C53BA1F1C63BA9F1C73BB1F1C83BB9F152
:10201000C93BC1F1CA3BC9F180E090E038C082EE13
:1020200090E035C089EE90E032C08AEE90E02FC09B
:1020300085EB90E02CC086EB90E029C087EB90E028
:1020400026C08CEC90E023C08DEC90E020C083E8AB
:1020500091E01DC08AE891E01AC082E991E017C0C2
:1020600084E991E014C081E292E011C083E292E041
:102070000EC084E292E00BC085E292E008C086E2E6
:1020800092E005C087E292E002C08AE292E0CF913E
:102090000C94940ECF910895882309F44BC0823894
:1020A00059F40E945C0E81FF45C089E30E94F61836
:1020B0000E94AE1989E30CC0833871F40E945C0E53
:1020C00080FF38C083E50E94F6180E94AE1983E5B0
:1020D0000E9435190C94AE19843859F40E945C0E94
:1020E00082FF28C087E40E94F6180E94AE1987E498
:1020F000EFCF9CEF980F913A58F390E2980F9830F9
:1021000050F4877091E001C0990F8A95EAF7892F02
:102110000E947D19DFCF9BE5980F933020F480E07B
:1021200090E00C947E0E885A833120F480E090E099
:102130000C94940E0895882321F00E9477190C9432
:10214000AE190895882321F00E947D190C94AE19D0
:102150000895BF92CF92DF92EF92FF920F931F9359
:10216000CF93DF9300D000D000D0CDB7DEB77C0195
:1021700085E0F701DE01119601900D928A95E1F755
:10218000F70183819481892B09F4DDC290818181DB
:102190008F3F19F49F3F09F4D6C2F70102812581D0
:1021A00022952F7099838A8389819A812E830E9438
:1021B000B518182FB92E0E94B4180E947B17EB2D6A
:1021C000E295EF704E2F50E0FA01E05AFF4F2E815A
:1021D0000C9499228B2D807F9B2D9F70F92E882344
:1021E00019F0F29480EFF822002349F0FF2009F45F
:1021F00057C28F2D0E9487190E94AE1951C2812F9C
:102200000E944C10FF2009F49EC28F2D0E948D1950
:1022100026960FB6F894DEBF0FBECDBFDF91CF91EB
:102220001F910F91FF90EF90DF90CF90BF900C9493
:10223000AE193B2D307F8B2D8F70303211F082958F
:10224000807F112319F0113021F12CC00023B9F047
:10225000222309F490C1213009F08DC126960FB6D2
:10226000F894DEBF0FBECDBFDF91CF911F910F91CC
:10227000FF90EF90DF90CF90BF900C94971922239E
:1022800019F0213009F45FC28E830E949A198E8161
:1022900086C1002321F0223008F055C26CC1211103
:1022A00052C27DC1002321F0222309F464C1F8C188
:1022B000222309F474C109C28B2D869586958370FB
:1022C00019F08130D1F03FC2002321F0812F9B2DE6
:1022D000937002C080E090E026960FB6F894DEBFBF
:1022E0000FBECDBFDF91CF911F910F91FF90EF9067
:1022F000DF90CF90BF900C947E0E002321F0812FB1
:102300009B2D937002C080E090E026960FB6F89463
:10231000DEBF0FBECDBFDF91CF911F910F91FF9018
:10232000EF90DF90CF90BF900C94940E812F0023FC
:1023300019F00E941D1D02C00E94851D26960FB631
:10234000F894DEBF0FBECDBFDF91CF911F910F91EB
:10235000FF90EF90DF90CF90BF900C940A1E8B2DD2
:10236000837009F075C00111EEC1812F82958695A9
:102370008770880F880F912F9F70C92ED12CE12C68
:10238000F12C082E04C0CC0CDD1CEE1CFF1C0A94A2
:10239000D2F714FF12C00FE010E020E030E004C0DC
:1023A000000F111F221F331F8A95D2F7C901B801F0
:1023B000609570958095909503C060E070E0CB01CA
:1023C0004B2D4695469543704230C1F060F56C291F
:1023D0007D298E299F29413051F126960FB6F89418
:1023E000DEBF0FBECDBFDF91CF911F910F91FF9048
:1023F000EF90DF90CF90BF900C94A2176C297D29AD
:102400008E299F2926960FB6F894DEBF0FBECDBF4A
:10241000DF91CF911F910F91FF90EF90DF90CF90C0
:10242000BF900C94BE170E94A217C701B601269652
:102430000FB6F894DEBF0FBECDBFDF91CF911F91D5
:102440000F91FF90EF90DF90CF90BF900C94861784
:10245000002319F08B2D817001C08695882309F423
:1024600072C1812F829586958770880F880F912F72
:102470009F70C92ED12CE12CF12C082E04C0CC0C5D
:10248000DD1CEE1CFF1C0A94D2F714FF12C00FE0F3
:1024900010E020E030E004C0000F111F221F331FA6
:1024A0008A95D2F7C901B80160957095809590958D
:1024B00003C060E070E0CB014B2D4695469543701C
:1024C0004230C1F060F56C297D298E299F29413069
:1024D00051F126960FB6F894DEBF0FBECDBFDF9147
:1024E000CF911F910F91FF90EF90DF90CF90BF9011
:1024F0000C947C186C297D298E299F2926960FB66D
:10250000F894DEBF0FBECDBFDF91CF911F910F9129
:10251000FF90EF90DF90CF90BF900C9498180E949E
:102520007C18C701B60126960FB6F894DEBF0FBE21
:10253000CDBFDF91CF911F910F91FF90EF90DF9072
:10254000CF90BF900C946018103FD1F118F4103E5A
:1025500050F4A1C0123F09F463C008F44CC0133F0B
:1025600009F473C098C01F708B2D8F710023A1F0E8
:102570000E94F917812F26960FB6F894DEBF0FBE82
:10258000CDBFDF91CF911F910F91FF90EF90DF9022
:10259000CF90BF900C949B100E941A18812F269602
:1025A0000FB6F894DEBF0FBECDBFDF91CF911F9164
:1025B0000F91FF90EF90DF90CF90BF900C94A210FE
:1025C0000023A9F02111BFC08B2D8F7126960FB665
:1025D000F894DEBF0FBECDBFDF91CF911F910F9159
:1025E000FF90EF90DF90CF90BF900C943F18223077
:1025F00008F0A9C0E9CF0023A9F08B2D8F71269692
:102600000FB6F894DEBF0FBECDBFDF91CF911F9103
:102610000F91FF90EF90DF90CF90BF900C94F9173F
:10262000002359F38B2D8F7126960FB6F894DEBFD9
:102630000FBECDBFDF91CF911F910F91FF90EF9013
:10264000DF90CF90BF900C941A18002399F08B2D37
:102650008F7126960FB6F894DEBF0FBECDBFDF9107
:10266000CF911F910F91FF90EF90DF90CF90BF908F
:102670000C94E41726960FB6F894DEBF0FBECDBFBC
:10268000DF91CF911F910F91FF90EF90DF90CF904E
:10269000BF900C94DA170023A9F0222309F4ADCFE0
:1026A000812F26960FB6F894DEBF0FBECDBFDF9107
:1026B000CF911F910F91FF90EF90DF90CF90BF903F
:1026C0000C94840F222309F4ADCF812F26960FB6E8
:1026D000F894DEBF0FBECDBFDF91CF911F910F9158
:1026E000FF90EF90DF90CF90BF900C944C104B2D4B
:1026F0004F70612FC7010E94AF0226960FB6F89463
:10270000DEBF0FBECDBFDF91CF911F910F91FF9024
:10271000EF90DF90CF90BF900C94FE164B2D4F7032
:10272000612FC70126960FB6F894DEBF0FBECDBF4E
:10273000DF91CF911F910F91FF90EF90DF90CF909D
:10274000BF900C94EF0526960FB6F894DEBF0FBE2F
:10275000CDBFDF91CF911F910F91FF90EF90DF9050
:10276000CF90BF9008950E9494190E9469190E9409
:10277000AE190E94BA1E0E940A1E80E090E00E94DC
:102780007E0E80E090E00C94940E0E9484190C94CC
:10279000B3130E94B518292F22952F702C3030F4D6
:1027A0002A3048F42250223078F405C02C3041F011
:1027B0002F3031F009C0803E48F0803F29F406C038
:1027C00093FB882780F9089580E0089581E00895BB
:1027D000CF93DF9300D000D01F92CDB7DEB70F901C
:1027E0000F900F900F900F90DF91CF910895CF939E
:1027F000DF9300D000D000D0CDB7DEB726960FB65D
:10280000F894DEBF0FBECDBFDF91CF9108951F9327
:10281000CF93DF93C091790116E080917A01C817B8
:1028200099F0D0E01C9FF0011D9FF00D1124E55898
:10283000FE4F4081518162817381848195810E9424
:10284000F7132196C770E9CFDF91CF911F910895BB
:102850004091AB015091AC016091AD017091AE011E
:102860008091AF019091B0010C94F7138091B00169
:1028700082958F7009F054C08091AD01882309F4CE
:102880004FC080917901A0917A014091AE015091A1
:10289000AF016091AB017091AC01B6E08A1709F409
:1028A0003FC090E041155105C1F17F3F11F46F3FEA
:1028B000A1F1B89FF001B99FF00D1124E558FE4F2A
:1028C000218127132AC02081261327C022812111AC
:1028D00024C0238134812417350710F42150310995
:1028E000241B350B283C3105C0F42091B0012F701A
:1028F00020612093B00126E0289FF001299FF00D70
:102900001124E058FE4F80818F70806180838BEAB4
:1029100091E00E94A9100C94071401968770BECF15
:102920000895CF92DF92EF92FF920F931F93CF9370
:10293000DF93CDB7DEB762970FB6F894DEBF0FBE58
:10294000CDBF8C0185E0F801DE011D9601900D924E
:102950008A95E1F7D8014C9111965C9111971296E6
:102960006C918091AE019091AF01009709F475C10F
:102970003091AB017091AC017F3F19F43F3F09F4F6
:102980006CC1F801C380D480E090AD01EE2009F461
:10299000BEC02091B001C816D90628F0D601A81BE8
:1029A000B90BCD0104C0809590958C0D9D1DFF2421
:1029B000F394883C910578F0F12C207F09F0C4C095
:1029C0007C2DD98AC88A89890E94E8138BEA91E014
:1029D0000E94A910AFC0822F807F09F045C0571315
:1029E00013C0431311C061110FC02F7020612093D9
:1029F000B0010E9428148BEA91E00E94A9108091F6
:102A0000B001F80185832EC0CD2819F15F3F11F484
:102A10004F3FF9F0F62E61111CC080917901209191
:102A20007A0136E0821709F45BC090E0389FF0012C
:102A3000399FF00D1124E558FE4F7181571306C0E0
:102A40007081471303C07281711103C001968770B2
:102A5000E9CFF62E662309F41CC18091B001816094
:102A60008093B001F12C15C1571309C0431307C05F
:102A7000611105C08091B001F8018583C8C04D8700
:102A80005E878D859E856A8B0E94C9136A8988231B
:102A9000D1F16623C1F12091B001822F82958F7010
:102AA00090E0029774F08091AB019091AC0198870F
:102AB0008F831986DB86CA862C87CE0107960E94F3
:102AC000A91086E0F801ABEAB1E001900D928A9579
:102AD000E1F70E9436140E942814FF24F394D9C011
:102AE0004D875E878D859E850E94B518292F22957A
:102AF0002F70223008F0C1C09F7009F0BBC0805E0B
:102B0000883008F4C6C0C8010E94A910E6CFC816D4
:102B1000D90608F453C0F601E81BF90BCF01883C35
:102B2000910508F450C0F12C7C2DD98AC88A898976
:102B30000E94E813EBEAF1E086E0DF011D928A953E
:102B4000E9F70E942814A5C0571314C0431312C0FC
:102B5000611110C08091B001F8018583C8010E9405
:102B6000A91086E0EBEAF1E0DF011D928A95E9F712
:102B7000FE2C8FC04D875E878D859E856A8B0E9457
:102B8000C9136A89882309F4BECF662309F4BBCF31
:102B90002091B001822F82958F7090E002970CF403
:102BA00090CF8091AB019091AC019A8389831B8275
:102BB000DD82CC822E83CE01019681CF80959095C7
:102BC0008C0D9D1DACCFF62E662309F49CCF5713B8
:102BD00033C0431331C02091B00120FD24C0822FA7
:102BE00082958F70482F50E041155105E1F0D801D2
:102BF00015962C9315974F30510549F08F5F982FFC
:102C00009295907F822F8F70892B15968C93C80197
:102C10000E94A91086E0F801ABEAB1E001900D92A4
:102C20008A95E1F78ECF86E0F801ABEAB1E001903A
:102C30000D928A95E1F72DC04D875E878D859E8523
:102C40000E94C91381113DCF8091B00181608093B2
:102C5000B001C8010E94A9101CC0662309F453CF1B
:102C60004D875E878D859E850E94C913882309F450
:102C70004ACF27CF811143CF0CC0243008F043CF77
:102C80009F7009F43CCFD80115969C91907F09F074
:102C900036CF8F2D62960FB6F894DEBF0FBECDBF34
:102CA000DF91CF911F910F91FF90EF90DF90CF9028
:102CB00008951F93CF93DF93CDB7DEB72C970FB650
:102CC000F894DEBF0FBECDBF4F83588769877A87E0
:102CD0008B879C87CE0107960E949114882371F000
:102CE0008A859B85892B09F441C088858F3F09F02F
:102CF00065C08F818F3F09F061C038C086E0FE015A
:102D00003796DE01119601900D928A95E1F76A855A
:102D10007B856115710551F1FF81E885EF3F11F465
:102D2000FF3F21F120917A0130E0C90101968770BF
:102D300099274091790150E08417950709F447C01D
:102D4000F983EA837D836C8396E0929FD001939F01
:102D5000B00D1124A558BE4FFE01319601900D9281
:102D60009A95E1F780937A010E94071416E080910A
:102D7000790190917A018917B9F1189FC001112446
:102D800085589E4F0E949114882371F1E09179013A
:102D90001E9FF0011124E558FE4F40815181628150
:102DA0007381848195810E94F7138091790190E06D
:102DB00001968770992780937901D9CF4F815885E3
:102DC00069857A858B859C850E94F713CFCF0E94F9
:102DD000C51310927A0110927901EBEAF1E086E0D6
:102DE000DF011D928A95E9F72C960FB6F894DEBFA5
:102DF0000FBECDBFDF91CF911F910895EF92FF924B
:102E00000F931F93CF93DF938C01892B09F46CC030
:102E1000F12CEE24E394E8012196F80184918437A3
:102E200040F4843008F051C0813081F0823019F1D3
:102E30005BC0853709F444C0A8F19CE7980F903730
:102E400008F052C08F770E944C1041C00E5F1F4F98
:102E5000FE01849190E2980F983050F48770FE2D17
:102E600001C0FF0F8A95EAF78F2F0E94871914C0BF
:102E70000E94840F2DC00E5F1F4FFE01849190E2CF
:102E8000980F983060F48770FE2D01C0FF0F8A956F
:102E9000EAF78F2F0E948D190E94AE1919C00E9467
:102EA0004C1016C00E5F1F4FFE01C491CC2381F061
:102EB0008FE99FE00197F1F700C00000C150F6CF05
:102EC0000E5F1F4FFE01F49003C00E94840F8E011D
:102ED0008F2D882309F49FCFEFE9FFE03197F1F7B9
:102EE00000C000008150F5CFDF91CF911F910F916D
:102EF000FF90EF90089508956093B5017093B60127
:102F00008093B7019093B8010C94B3130F931F9360
:102F10000091B5011091B6012091B7013091B8012F
:102F2000DC01CB01802B912BA22BB32B8093B5011D
:102F30009093B601A093B701B093B8011F910F9180
:102F40000C94B3130F931F930091B5011091B60128
:102F50002091B7013091B801DC01CB01802391238E
:102F6000A223B3238093B5019093B601A093B70138
:102F7000B093B8011F910F910C94B3130F931F934B
:102F80000091B5011091B6012091B7013091B801BF
:102F9000DC01CB0180279127A227B3278093B501BD
:102FA0009093B601A093B701B093B8011F910F9110
:102FB0000C94B3131092B1011092B2011092B301AC
:102FC0001092B4010C94B31341E050E060E070E063
:102FD00004C0440F551F661F771F8A95D2F7409390
:102FE000B1015093B2016093B3017093B4010C949A
:102FF000B31341E050E060E070E004C0440F551F9F
:10300000661F771F8A95D2F78091B1019091B20126
:10301000A091B301B091B401482B592B6A2B7B2BA3
:103020004093B1015093B2016093B3017093B40126
:103030000C94B31341E050E060E070E004C0440F32
:10304000551F661F771F8A95D2F74095509560955A
:1030500070958091B1019091B201A091B301B091AE
:10306000B401482359236A237B234093B101509331
:10307000B2016093B3017093B4010C94B31341E0B7
:1030800050E060E070E004C0440F551F661F771FDA
:103090008A95D2F78091B1019091B201A091B301CC
:1030A000B091B401482759276A277B274093B10183
:1030B0005093B2016093B3017093B4010C94B313B5
:1030C0000F931F930091B1011091B2012091B301B0
:1030D0003091B401DC01CB01802B912BA22BB32BBF
:1030E0008093B1019093B201A093B301B093B40166
:1030F0001F910F910C94B3130F931F930091B10183
:103100001091B2012091B3013091B401DC01CB01E7
:1031100080239123A223B3238093B1019093B20122
:10312000A093B301B093B4011F910F910C94B3130A
:103130000F931F930091B1011091B2012091B3013F
:103140003091B401DC01CB0180279127A227B3275E
:103150008093B1019093B201A093B301B093B401F5
:103160001F910F910C94B3130895CF92DF92EF92B9
:10317000FF920F931F93CF93DF938C01C090B10107
:10318000D090B201E090B301F090B4018091B5010C
:103190009091B601A091B701B091B801C82AD92A7F
:1031A000EA2AFB2ACFE1D0E0D701C6010C2E04C0E9
:1031B000B695A795979587950A94D2F780FF07C093
:1031C000B8018C2F0E9413068130910531F42197AC
:1031D00058F7B80180E00E941306DF91CF911F914C
:1031E0000F91FF90EF90DF90CF90089590910C0198
:1031F0009923F1F090910D019923D1F0982F969594
:10320000969596959F3080F5E0910E01F0910F0113
:10321000E90FF11D877021E030E0A90102C0440FE1
:10322000551F8A95E2F7CA019181892B8183089500
:1032300020910E0130910F01F90132969FEF40E08D
:103240005191851789F09F3F19F4511101C0942FB6
:103250004F5F4E30A9F79F3F39F0F901E90FF11D9B
:1032600097FDFA9582830895089590910C01992312
:10327000F9F090910D019923D9F0982F9695969594
:1032800096959F3028F5E0910E01F0910F01E90F1E
:10329000F11D877021E030E0A90102C0440F551FE5
:1032A0008A95E2F7CA0180959181892381830895E7
:1032B00020910E0130910F01F9013296205F3F4FAE
:1032C0009081891301C010823196E217F307C1F78C
:1032D000089581E090E0E0910E01F0910F01E80F78
:1032E000F91F1082019680319105A9F708959091F8
:1032F000CB01892B8093CB01089580959091CB01D0
:1033000089238093CB0108951092CB010895909169
:10331000CA01892B8093CA01089580959091CA01B2
:1033200089238093CA0108951092CA010895809359
:10333000B90108951092B901089580910E019091FC
:103340000F01FC0131969C01205F3F4F80E091917D
:1033500091118F5FE217F307D1F70895E0910E0105
:10336000F0910F018091CB018083E0910E01F091EB
:103370000F0190818091CA01892B80838091B901CE
:10338000882361F0E0910E01F0910F019081892B6B
:1033900080830E949D1981111092B90180910E01C4
:1033A00090910F010C94680ECF92DF92EF92FF92F2
:1033B0006C01EE24FF24C114D104E104F10421F0D6
:1033C000C701B60120E101C020E0C72ED82EE92EAA
:1033D000FF24C114D104E104F10419F0285FC701EE
:1033E000B6016B017C0154E0F694E794D794C7943E
:1033F0005A95D1F7C114D104E104F10419F02C5FFE
:10340000C701B6016B017C0142E0F694E794D794C2
:10341000C7944A95D1F7C114D104E104F10419F01D
:103420002E5FC701B601DC01CB01B695A795979534
:103430008795892B8A2B8B2B09F02F5F822FFF908A
:10344000EF90DF90CF9008958091E401843011F1E6
:1034500020E488E190E00FB6F894A895809360008E
:103460000FBE2093600083B7817F846083BF83B7E2
:10347000816083BF7894889583B78E7F83BF0FB6B2
:10348000F894A89580916000886180936000109204
:1034900060000FBE089508950C944B1ACF930E94BC
:1034A0004C1A0E9432040E944B1AC0E08C2F0E94DA
:1034B0002805811104C0CF5FCE30C1F701C081E083
:1034C000CF9108950E94C5130E945C0E0C94520780
:1034D00082E084BD93E095BD9AEF97BD80936E0026
:1034E00008952FB7F8948091CD019091CE01A091CD
:1034F000CF01B091D0012FBF0895CF92DF92EF920C
:10350000FF920F931F932FB7F8944091CD015091E4
:10351000CE016091CF017091D0012FBF6A017B0174
:10352000EE24FF248C0120E030E0C016D106E20634
:10353000F30610F4415051099A01281B390BC901B7
:103540001F910F91FF90EF90DF90CF9008951F9201
:103550000F920FB60F9211248F939F93AF93BF9347
:103560008091CD019091CE01A091CF01B091D00179
:103570000196A11DB11D8093CD019093CE01A09322
:10358000CF01B093D001BF91AF919F918F910F90D8
:103590000FBE0F901F9018950E94540BF8942FEFB8
:1035A00087EA91E6215080409040E1F700C000009A
:1035B00087E090EBDC018093ED019093EE01A09306
:1035C000EF01B093F0019CE088E10FB6F894A89564
:1035D000809360000FBE90936000FFCFEF92FF9248
:1035E0000F931F93CF93DF93D82FC0E08C2F0E94AF
:1035F000280500E010E0E82EF12CC701002E02C0E3
:10360000959587950A94E2F780FD06C00F5F1F4FDE
:103610000630110591F709C0602F7C2F80E00E94D1
:10362000F0058D13F3CF81E004C0CF5FCE30F1F60B
:1036300080E0DF91CF911F910F91FF90EF9008955F
:10364000CF93C82F8CE20E94EE1A882321F08C2F92
:10365000CF910C94EE1A80E0CF910895CF930E9401
:10366000751C811102C00E945B1CC5E6C15049F067
:103670000E9432048FE39CE90197F1F700C000003B
:10368000F5CF89E20E94201B811113C18AE20E94BA
:10369000201B81110E945B1C85E00E94201B811170
:1036A0000E94CC1A0E94801C8093CC0187E00E946B
:1036B000201B8823A9F18BE10E94201B882351F055
:1036C0008091CC0181FB222720F991E0922790FB89
:1036D00081F90EC08EE00E94201B882361F080914A
:1036E000CC0182FB222720F991E0922790FB82F9FE
:1036F0008093CC0115C080E10E94201B9091CC01E9
:10370000882341F093FB222720F981E0822780FB68
:1037100093F904C0892F809580FB90F99093CC0198
:103720008091CC010E94841C0E94921C8093DE0137
:1037300080EE0E94201B882341F08091DE01982FAB
:10374000909590FB80F98093DE0189E30E94201B15
:10375000882359F08091DE0181FB222720F991E036
:10376000922790FB81F98093DE0182EE0E94201B5C
:10377000882359F08091DE0182FB222720F991E015
:10378000922790FB82F98093DE0186EE0E94201B37
:10379000882359F08091DE0183FB222720F991E0F4
:1037A000922790FB83F98093DE0183EE0E94201B19
:1037B000882359F08091DE0184FB222720F991E0D3
:1037C000922790FB84F98093DE0185E30E94201B01
:1037D000882359F08091DE0185FB222720F991E0B2
:1037E000922790FB85F98093DE0181E30E94201BE4
:1037F000882359F08091DE0186FB222720F991E091
:10380000922790FB86F98093DE0181E10E94201BC4
:10381000882359F08091DE0187FB222720F991E06F
:10382000922790FB87F98093DE018091DE010E9450
:10383000961C8091DE0187FB882780F980930D011B
:1038400087E20E94201BC82F8EE10E94201B81115D
:10385000C2608FE10E94201B8111C46080E20E943F
:10386000201B8111C86081E20E94201B8111C06170
:1038700082E20E94201B8111C06283E20E94201B11
:103880008111C06484E20E94201B882311F0C0686B
:1038900002C0CC2329F08C2F0E948D1C6C2F03C0FA
:1038A0000E94891C682F70E080E090E0CF910C941A
:1038B0007C17CF9108956DEE7EEF80E090E00E943E
:1038C000CF2260E082E090E00E94C12260E083E0CD
:1038D00090E00E94C12260E084E090E00E94C1225A
:1038E00060E085E090E00C94C12280E090E00E94CE
:1038F000BB2221E08D3E9E4F09F020E0822F0895EB
:1039000082E090E00C94B322682F82E090E00C9467
:10391000C12283E090E00C94B322682F83E090E012
:103920000C94C12284E090E00C94B322682F84E0D0
:1039300090E00C94C1228091D30180FF0BC0609174
:10394000130185E0689FB001112475956795759501
:1039500067952BC081FF09C06091130185E0689FC6
:10396000B00111247595679520C082FF07C0609152
:10397000130185E0689FB001112417C09091D40114
:103980009923D1F060911201961788F720911301C5
:1039900085E0289F90011124929FA001939F500DD4
:1039A000112470E0CA010E9485226038710540F43C
:1039B0006115710519F406C065E070E0862F089561
:1039C0008FE7089581E008958091D30180FF08C0BA
:1039D0006091110170E0759567957595679521C0A7
:1039E00081FF06C06091110170E07595679519C05F
:1039F00082FF04C06091110170E010C09091D40169
:103A0000992399F0609110019617A0F78091110108
:103A1000899FC001112470E00E94852260387105E1
:103A200040F46115710519F406C061E070E0862F5D
:103A300008958FE7089581E00895803F21F40E9462
:103A40009B1C819504C0813F29F40E949B1C80939C
:103A5000D7010895823F21F40E949B1C819504C0E8
:103A6000833F29F40E949B1C8093D6010895893FCF
:103A700019F40E94E41C05C08A3F31F40E94E41C42
:103A800081958093D80108958B3F21F40E94E41C16
:103A9000819504C08C3F29F40E94E41C8093D901D5
:103AA0000895843F21F48091D501816017C0853F3E
:103AB00021F48091D501826011C0863F21F480916C
:103AC000D50184600BC0873F21F48091D5018860C7
:103AD00005C0883F31F48091D50180618093D50184
:103AE00008958D3F21F48091D30181600BC08E3FFA
:103AF00021F48091D301826005C08F3F29F4809129
:103B0000D30184608093D3010895803F39F480917C
:103B1000D70187FF6CC01092D70169C0813F29F49B
:103B20008091D7011816BCF362C09091D601823FF4
:103B300029F497FF5CC01092D60159C0833F19F455
:103B40001916CCF354C0893F41F48091D80118165E
:103B50000CF04DC01092D8014AC08A3F29F48091E0
:103B6000D80187FF44C0F6CF8B3F39F48091D9014B
:103B700087FF3DC01092D9013AC08C3F29F4809153
:103B8000D9011816BCF333C0843F21F48091D501CC
:103B90008E7F17C0853F21F48091D5018D7F11C0A4
:103BA000863F21F48091D5018B7F0BC0873F21F4A4
:103BB0008091D501877F05C0883F31F48091D50180
:103BC0008F7E8093D50113C08D3F21F48091D30166
:103BD0008E7F0BC08E3F21F48091D3018D7F05C075
:103BE0008F3F29F48091D3018B7F8093D301809103
:103BF000D60181110EC08091D70181110AC0809138
:103C0000D801811106C08091D901811102C01092A2
:103C1000D401089585ED91E00E94730E0E94711AFF
:103C20009093D2018093D10108951F93CF93DF9396
:103C30008091D1019091D2010E947D1AAC019091A6
:103C4000D401992321F02091140130E006C0209185
:103C500015018AE0289F900111244217530708F4A8
:103C600085C08091D601C091D701D091D801109123
:103C7000D901811107C0C11175C0D11173C01111D3
:103C800071C074C09F3F19F09F5F9093D4011816C4
:103C900024F40E949B1C8093D6018091D60187FF5B
:103CA00005C00E949B1C81958093D6011C1624F4AC
:103CB0000E949B1C8093D7018091D70187FF05C08C
:103CC0000E949B1C81958093D7016091D601662349
:103CD00031F1C091D701CC2311F1062E000C770BE6
:103CE000880B990B0E948C2123E333E343E35FE3CA
:103CF0000E94F0210E9454216093D6016C2FCC0FBA
:103D0000770B880B990B0E948C2123E333E343E369
:103D10005FE30E94F0210E9454216093D7011D1699
:103D200024F40E94E41C8093D8018091D80187FF7D
:103D300005C00E94E41C81958093D801111624F4DB
:103D40000E94E41C8093D9018091D90187FF05C0AE
:103D50000E94E41C81958093D901DF91CF911F913E
:103D60000C940A1E9F3F09F08FCFA0CFDF91CF9117
:103D70001F910895E5EDF1E085E0DF011D928A9540
:103D8000E9F71092D4011092D3010895833081F1A4
:103D900028F4813059F08230D1F00895853009F44B
:103DA00049C0B8F1863009F456C0089580911501D4
:103DB000262F30E0280F311D2F3F310524F4680FE6
:103DC0006093150108958FEF8093150108958091F8
:103DD0001401262F30E0280F311D2F3F310524F428
:103DE000680F6093140108958FEF80931401089574
:103DF00080911301262F30E0280F311D2F3F310510
:103E000024F4680F6093130108958FEF80931301DA
:103E1000089580911201262F30E0280F311D2F3F89
:103E2000310524F4680F6093120108958FEF809399
:103E30001201089580911101262F30E0280F311DC5
:103E40002F3F310524F4680F6093110108958FEF1F
:103E500080931101089580911001262F30E0280FE2
:103E6000311D2F3F310524F4680F60931001089530
:103E70008FEF809310010895833011F128F4813081
:103E800049F0823091F00895853081F120F186303B
:103E9000C1F1089580911501681720F4861B809365
:103EA0001501089510921501089580911401681765
:103EB00020F4861B80931401089510921401089534
:103EC00080911301681720F4861B809313010895D5
:103ED00010921301089580911201681720F4861B37
:103EE000809312010895109212010895809111019A
:103EF000681720F4861B8093110108951092110118
:103F0000089580911001681720F4861B809310019A
:103F100008951092100108950F931F938D3109F4A5
:103F20006BC008F03FC08E3009F47DC0C0F487300C
:103F300009F46EC068F4863009F0AFC08091CC01FE
:103F4000817F8E7F8093CC0181E08093DB01A6C0CE
:103F5000883009F458C08B3009F49BC09EC086316C
:103F600009F497C078F4803109F470C0813109F008
:103F700094C00E94C51390910D0181E08927809320
:103F80000D0187C0893109F484C08B3109F085C0E7
:103F90008091CC0181FB222720F991E0922790FBB0
:103FA00081F94AC0853309F45BC048F4873209F4CB
:103FB00057C008F45AC0893209F452C06EC0833425
:103FC00038F48A3308F067C0883309F462C065C0EA
:103FD000833409F445C0883409F05FC00E94C513DA
:103FE0000FEF13ED20E3015010402040E1F700C037
:103FF00000000E94CC1A4DC00E940E210E945C0E4F
:104000000E94520746C00E94801C0E94921C41C020
:104010009091CC01892F817090FF12C0917F9E7F7B
:104020009093CC013BC08091CC0182FB222720F9E8
:1040300091E0922790FB82F98093CC01992349F17A
:104040008091CC0181608093CC0123C08091CC0110
:1040500083FB222720F991E0922790FB83F9ECCF94
:1040600061E070E080E090E010C08D5141E050E0F0
:1040700060E070E08A019B0104C0000F111F221F45
:10408000331F8A95D2F7C901B8010E947C170E949C
:10409000C51381E003C08953E9CF80E01F910F91E0
:1040A000089580E008950C945120CF93C82F8091FB
:1040B000DB01813079F018F08230E9F187C0E091BE
:1040C0000E01F0910F018081813169F0823209F097
:1040D0007FC009C0E0910E01F0910F018081813114
:1040E00011F0823261F48C2F0E945320811104C0A0
:1040F0008C2F0E948C1F1DC081E090E01AC08C2F75
:104100000E945120811114C0C43179F048F4CB30A1
:1041100079F0C03109F060C082E08093DB0108C013
:10412000C93219F0C83321F057C01092DB0154C0D6
:1041300081E0817053C0C93289F118F5C43171F141
:10414000A8F4C73009F046C08AE08093150194E1D5
:104150009093140193E0909313018093120188E0EF
:104160008093110188E28093100134C0CE51C63093
:1041700088F5EC2FF0E0E65DFE4F80818093DA0158
:1041800029C0CE34E9F020F4CB3421F56AE013C025
:10419000C13579F0C235F1F461E00DC08091DA01EA
:1041A000882319F01092DA0115C081E08093DB01B9
:1041B00015C061E006C08091DA010E94C61E0AC0E7
:1041C0006AE08091DA010E943C1F04C01092DB017A
:1041D00080E004C081E002C080E0ABCFCF910895C1
:1041E000E1E8F0E080818860808380818160808365
:1041F0008FB7F89493E09093890090ED90938800A6
:104200008FBF0895EFE6F0E080818260808308959B
:10421000EFE6F0E080818D7F80830895EFE6F0E0A7
:10422000908182E08927808308951F920F920FB6B4
:104230000F9211242F933F934F935F936F937F932C
:104240008F939F93AF93BF93EF93FF938091DC0184
:104250009091DD0101969093DD018093DC01811145
:1042600003C082E00E945207E091DD01E695E695E9
:10427000F0E0E457FB4FE4918091DC018E1303C022
:1042800080E00E945207FF91EF91BF91AF919F9103
:104290008F917F916F915F914F913F912F910F90EF
:1042A0000FBE0F901F9018950E945B216894B1116A
:1042B0000C94EA2108950E94CF2188F09F5798F02E
:1042C000B92F9927B751B0F0E1F0660F771F881F1B
:1042D000991F1AF0BA95C9F714C0B13091F00E9435
:1042E000E921B1E008950C94E921672F782F882700
:1042F000B85F39F0B93FCCF3869577956795B3955C
:10430000D9F73EF490958095709561957F4F8F4FCA
:104310009F4F0895E89409C097FB3EF490958095CF
:10432000709561957F4F8F4F9F4F9923A9F0F92F7B
:1043300096E9BB279395F695879577956795B795F9
:10434000F111F8CFFAF4BB0F11F460FF1BC06F5FDF
:104350007F4F8F4F9F4F16C0882311F096E911C0F1
:10436000772321F09EE8872F762F05C0662371F012
:1043700096E8862F70E060E02AF09A95660F771F26
:10438000881FDAF7880F9695879597F9089557FD56
:104390009058440F551F59F05F3F71F04795880FB3
:1043A00097FB991F61F09F3F79F08795089512164A
:1043B00013061406551FF2CF4695F1DF08C01616F6
:1043C00017061806991FF1CF8695710561050894A7
:1043D0000895E894BB2766277727CB0197F90895BE
:1043E0000E9403220C9474220E94662238F00E94DC
:1043F0006D2220F0952311F00C945D220C94632221
:1044000011240C94EA210E94C72170F3959FC1F3F7
:10441000950F50E0551F629FF001729FBB27F00D72
:10442000B11D639FAA27F00DB11DAA1F649F6627C7
:10443000B00DA11D661F829F2227B00DA11D621F16
:10444000739FB00DA11D621F839FA00D611D221FD0
:10445000749F3327A00D611D231F849F600D211DB4
:10446000822F762F6A2F11249F5750409AF0F1F037
:1044700088234AF0EE0FFF1FBB1F661F771F881FA0
:1044800091505040A9F79E3F510580F00C945D2259
:104490000C94EA215F3FE4F3983ED4F38695779538
:1044A0006795B795F795E7959F5FC1F7FE2B880F46
:1044B000911D9695879597F9089597F99F6780E8DC
:1044C00070E060E008959FEF80EC089500240A9466
:1044D0001616170618060906089500240A941216DF
:1044E0001306140605060895092E0394000C11F412
:1044F000882352F0BB0F40F4BF2B11F460FF04C0BF
:104500006F5F7F4F8F4F9F4F089597FB072E16F4D5
:10451000009407D077FD09D00E949F2207FC05D0A8
:104520003EF4909581959F4F0895709561957F4FCA
:104530000895EE0FFF1F0590F491E02D0994AA1B3A
:10454000BB1B51E107C0AA1FBB1FA617B70710F07E
:10455000A61BB70B881F991F5A95A9F780959095B0
:10456000BC01CD010895F999FECF92BD81BDF89AA5
:10457000992780B50895A8E1B0E042E050E00C949E
:10458000D622262FF999FECF1FBA92BD81BD20BD3C
:104590000FB6F894FA9AF99A0FBE019608950E9400
:1045A000C122272F0C94C222DC01CB01FC01F99916
:1045B000FECF06C0F2BDE1BDF89A319600B40D926F
:0C45C00041505040B8F70895F894FFCF28
:1045CC0020025307E307BE078A0756070101BA0109
:1045DC0028080A03140A3F4D36394D040004CA0357
:1045EC00910324033D0356036F03010203040506E4
:0445FC0007080900A3
:00000001FF
